:020000040000FA
:0A0000000000000025EF00F03FD0E3
:080018008CD00B6A0A6EFF0E8A
:100020000A260B2200D0D8A01200030E096EE60E9D
:1000300002D8F5D7096AFE0F086EE86A095AD8A0F7
:1000400012000000080600D0F8D7006A4F0EAF6E0D
:10005000240EAC6E900EAB6E00010FEE7FF0ED6AD9
:10006000E950EA10FCE1EF6A0F0EC16E070EB46EA4
:10007000C69AC30E926EE00E936EC00E946E92807E
:100080009282949294946ED0F2A403D0F294817AE6
:1000900011009EAA19D0060EAB1412E1E2CF29F08E
:1000A000E1CF28F02A2A10EE6BF02A50E126000E4C
:1000B000E222AECFE7FF29C0E2FF28C0E1FF110036
:1000C000AE50AE50AB98AB8811002A502B5C14E0B8
:1000D0002B2AEACF09F0E9CF08F000EE6BF02B50A5
:1000E000E926000EEA22EF50086E09C0EAFF08C0B8
:1000F000E9FFD880120004D0E868086ED8A012008A
:1001000012002A6A2B6A9D8A9F8AF28EF28C120054
:100110009D9A00EE6BF0010EF46EF36AF306000E8A
:10012000F45AEE6AF450F310F9E12A6A2B6A9D8AB8
:100130001200F29EE0CF6BF9D8CF6CF9E8CF6DF9E1
:10014000F28E0001A192B36AB26AF29E6BC9E0FF1F
:100150006CC9D8FF6DC9E8FFF28E10009EA8FED7CB
:10016000AD6E1200040ECA6ECB68BB6A0C0EBA6E7E
:100170009492040ECA6ECB68BE6A0C0EBD6E949447
:10018000CF0EBA16000EBA12000EBB6ECF0EBD1601
:10019000000EBD12000EBE6E939A8A8A320E3DDFAB
:1001A000939A8A9A92988998929A899A93948A941F
:1001B000949A8B9A93908A9093928A9294968B9623
:1001C00094988B9894908B9093968A9693988A980B
:1001D00092968996206A276800EE43F0240EEE6816
:1001E000E82EFDD71F6A8DDF93DFCD6AF294F28A85
:1001F000870ED56EB16AA192A082B36AB26AD08E20
:10020000A292B10EB16EA8EC07F0A9EC0BF010ECC5
:100210000EF0010E3E6EB60EA1DF420E9FDF000E05
:100220009DDF252AE86A25B2010F26B0010806E104
:1002300026703F2A000E40224122422246DF106EE5
:10024000B70E105C07E3FE0E105C01E301D0126AEA
:1002500085EF05F010AE22D0126A860E105C05E123
:1002600010C012F01368146817D0960E105C05E1E8
:1002700010C012F0156816680FD0A60E105C05E1CC
:1002800010C012F01768186807D0B60E105C04E1B1
:1002900010C012F019681A6884EF05F0125204E1D8
:1002A00085EF05F084EF05F0860E125CD8A4D0D05F
:1002B000132803E110C013F0C7D010C014F0180EBB
:1002C000135C0AE1860E4ADF135048DF145046DF04
:1002D000136885EF05F0B5D0220E135C0DE32F0EE9
:1002E000135C0AE2860E3ADF135038DF145036DF13
:1002F000136885EF05F0A5D0410E135C0DE3480EA1
:10030000135C0AE2860E2ADF135028DF145026DF22
:10031000136885EF05F095D0480E135C0AE1860E50
:100320001DDF13501BDF145019DF136885EF05F034
:1003300088D04D0E135C0AE1860E10DF13500EDFDD
:1003400014500CDF136885EF05F07BD05F0E135C53
:100350000AE1860E03DF135001DF1450FFDE13683D
:1003600085EF05F06ED03A0E135C07E18998209076
:10037000466845684468436864D03B0E135C07E1F7
:10038000899A20924A684968486847685AD0190E85
:10039000135C07E18B9620944E684D684C684B685F
:1003A00050D01A0E135C07E18B9820965268516862
:1003B00050684F6846D01B0E135C07E18B90209865
:1003C00056685568546853683CD07A0E135C07E150
:1003D0008B9A209A5A6859685868576832D0780EB4
:1003E000135C07E18A90209C5E685D685C685B68CE
:1003F00028D0790E135C07E18A92209E62686168BA
:1004000060685F681ED0150E135C0BE1CF0EBA1644
:10041000000EBA12000EBB6E666865686468636899
:1004200010D07B0E135C0AE1CF0EBD16000EBD127C
:10043000000EBE6E136885EF05F003D0136885EFDC
:1004400005F0136884EF05F085EF05F084EF05F003
:10045000960E125CD8A433EF05F0152804E110C005
:1004600015F031EF05F010C016F01652D8A4C7D021
:10047000180E155C0AE1860E71DE15506FDE000E57
:100480006DDE156885EF05F0B5D0220E155C0DE325
:100490002F0E155C0AE2860E61DE15505FDE000E3F
:1004A0005DDE156885EF05F0A5D0410E155C0DE306
:1004B000480E155C0AE2860E51DE15504FDE000E26
:1004C0004DDE156885EF05F095D0480E155C0AE104
:1004D000860E44DE155042DE000E40DE156885EFC4
:1004E00005F088D04D0E155C0AE1860E37DE1550FA
:1004F00035DE000E33DE156885EF05F07BD05F0E2C
:10050000155C0AE1860E2ADE155028DE000E26DE76
:10051000156885EF05F06ED03A0E155C07E18998F5
:100520002090466845684468436864D03B0E155C7B
:1005300007E1899A20924A684968486847685AD012
:10054000190E155C07E18B9620944E684D684C6837
:100550004B6850D01A0E155C07E18B9820965268B4
:10056000516850684F6846D01B0E155C07E18B90B0
:10057000209856685568546853683CD07A0E155CCC
:1005800007E18B9A209A5A6859685868576832D0A0
:10059000780E155C07E18A90209C5E685D685C6857
:1005A0005B6828D0790E155C07E18A92209E62680C
:1005B000616860685F681ED0150E155C0BE1CF0E98
:1005C000BA16000EBA12000EBB6E666865686468E3
:1005D000636810D07B0E155C0AE1CF0EBD16000ECD
:1005E000BD12000EBE6E156885EF05F003D01568CC
:1005F00085EF05F0156884EF05F031EF05F0180E72
:10060000155C0EE1960EAEEC00F01550AEEC00F06D
:100610001650AEEC00F0156885EF05F02FEF05F0F1
:10062000220E155C10E32F0E155C0DE2960EAEEC5B
:1006300000F01550AEEC00F01650AEEC00F015686E
:1006400085EF05F00CD2410E155C10E3480E155CE9
:100650000DE2960EAEEC00F01550AEEC00F0165028
:10066000AEEC00F0156885EF05F0F9D1480E155C89
:100670000DE1960EAEEC00F01550AEEC00F0165009
:10068000AEEC00F0156885EF05F0E9D14D0E155C74
:100690000DE1960EAEEC00F01550AEEC00F01650E9
:1006A000AEEC00F0156885EF05F0D9D15F0E155C52
:1006B0000DE1960EAEEC00F01550AEEC00F01650C9
:1006C000AEEC00F0156885EF05F0C9D13A0E155C67
:1006D00039E108EE6BF0D8901634E926000EEA22D4
:1006E000EECF2CF0EFCF2DF02E6A2F6A07EE6BF0D5
:1006F000D8901634E926000EEA22EECF30F0EFCF84
:1007000031F0326A336A7D0E165C06E389884668EA
:1007100045684468436815D089882C503F24026E90
:100720002D504020036E2E504120046E2F50422049
:10073000056E05C046F004C045F003C044F002C099
:1007400043F08DD13B0E155C39E108EE6BF0D8908B
:100750001634E926000EEA22EECF34F0EFCF35F062
:10076000366A376A07EE6BF0D8901634E926000E29
:10077000EA22EECF38F0EFCF39F03A6A3B6A7D0ECD
:10078000165C06E3898A4A6849684868476815D054
:10079000898A34503F24026E35504020036E365013
:1007A0004120046E37504220056E05C04AF004C057
:1007B00049F003C048F002C047F051D1190E155C52
:1007C00021E18B8602EE6BF0D8901634E926000EFC
:1007D000EA22EECF06F0EFCF07F006503F24026E7C
:1007E00007504020036E000E4120046E000E422090
:1007F000056E05C04EF004C04DF003C04CF002C0C1
:100800004BF02DD11A0E155C21E18B8802EE6BF0B6
:10081000D8901634E926000EEA22EECF06F0EFCF8C
:1008200007F006503F24026E07504020036E000E72
:100830004120046E000E4220056E05C052F004C037
:1008400051F003C050F002C04FF009D11B0E155CEF
:1008500021E18B8004EE6BF0D8901634E926000E6F
:10086000EA22EECF06F0EFCF07F006503F24026EEB
:1008700007504020036E000E4120046E000E4220FF
:10088000056E05C056F004C055F003C054F002C018
:1008900053F0E5D07A0E155C2DE116C022F08B8A5C
:1008A0007F0E225C21E2208A06EE6BF0D890223483
:1008B000E926000EEA22EECF06F0EFCF07F0065051
:1008C0003F24026E07504020036E000E4120046E4C
:1008D000000E4220056E05C05AF004C059F003C056
:1008E00058F002C057F005D0209A5A6859685868E5
:1008F0005768B5D0780E155C2DE116C023F08A80BC
:100900007F0E235C21E2208C06EE6BF0D89023341E
:10091000E926000EEA22EECF06F0EFCF07F00650F0
:100920003F24026E07504020036E000E4120046EEB
:10093000000E4220056E05C05EF004C05DF003C0ED
:100940005CF002C05BF005D0209C5E685D685C686E
:100950005B6885D0790E155C2DE116C024F08A8283
:100960007F0E245C21E2208E06EE6BF0D8902434BA
:10097000E926000EEA22EECF06F0EFCF07F0065090
:100980003F24026E07504020036E000E4120046E8B
:10099000000E4220056E05C062F004C061F003C085
:1009A00060F002C05FF005D0209E626861686068F8
:1009B0005F6855D0150E155C2FE13D6A16C03CF0FE
:1009C000D8903C363D363C363D3602EE6BF0D89042
:1009D0003E34E926000EEA22EECF06F0EFCF07F014
:1009E00006503F24026E07504020036E000E412047
:1009F000046E000E4220056E05C066F004C065F06E
:100A000003C064F002C063F0CF0EBA16300EBA1203
:100A1000FF0EBB6E156823D07B0E155C1EE13D6A90
:100A200016C03CF0D8903C363D363C363D363C3620
:100A30003D36070E3C26000E3D2200EE3CF0CF0E68
:100A4000BD16EE38300BBD12ED30F36EEF30BE6EDA
:100A5000F332BE32156859D002D0156856D01568E9
:100A600053D053D051D0A60E125C0BE1172803E1EE
:100A700010C017F004D010C018F0BFD945D045D031
:100A800043D0B60E125C20E1192803E110C019F022
:100A900019D010C01AF01E0E195C09E0420E195C44
:100AA00006E0470E195C03E07B0E195C09E1B60E07
:100AB000AEEC00F01950AEEC00F01A50AEEC00F0C5
:100AC000E5D922D022D020D0C60E125C07E11B2827
:100AD00003E110C01BF01B6818D016D0D60E125CB4
:100AE00007E11C2803E110C01CF01C680ED00CD0DC
:100AF000E60E125C09E11D2803E110C01DF003D0D1
:100B000010C01EF01D6801D03ED9090E275CD8B078
:100B100031D167503F5C68504058695041586A5025
:100B20004258D8A019D16A8E27522EE18078929827
:100B300080B815D030503F24026E31504020036EF3
:100B400032504120046E33504220056E05C046F0FD
:100B500004C045F003C044F002C043F014D02C5050
:100B60003F24026E2D504020036E2E504120046E13
:100B70002F504220056E05C046F004C045F003C06A
:100B800044F002C043F0E7D0010E275C2EE1807AEA
:100B9000929A80BA15D038503F24026E39504020C6
:100BA000036E3A504120046E3B504220056E05C052
:100BB0004AF004C049F003C048F002C047F014D026
:100BC00034503F24026E35504020036E3650412091
:100BD000046E37504220056E05C04AF004C049F04B
:100BE00003C048F002C047F0B6D0020E275C06E111
:100BF0008B964E684D684C684B68ADD0030E275CF1
:100C000006E18B985268516850684F68A4D0040E72
:100C1000275C06E18B9056685568546853689BD0F2
:100C2000050E275C2AE120BA06D08B9A5A685968CB
:100C30005868576821D0827A949A06EE6BF0D89063
:100C40002234E926000EEA22EECF06F0EFCF07F0BD
:100C500006503F24026E07504020036E000E4120D4
:100C6000046E000E4220056E05C05AF004C059F013
:100C700003C058F002C057F06ED0060E275C2AE180
:100C800020BC06D08A905E685D685C685B6821D095
:100C90008170939006EE6BF0D8902334E926000E15
:100CA000EA22EECF06F0EFCF07F006503F24026EA7
:100CB00007504020036E000E4120046E000E4220BB
:100CC000056E05C05EF004C05DF003C05CF002C0BC
:100CD0005BF041D0070E275C2AE120BE06D08A9245
:100CE0006268616860685F6821D08172939206EEE5
:100CF0006BF0D8902434E926000EEA22EECF06F0FD
:100D0000EFCF07F006503F24026E07504020036EDD
:100D1000000E4120046E000E4220056E05C062F0F8
:100D200004C061F003C060F002C05FF014D0080E90
:100D3000275C11E1666865686468636800EE3CF0F2
:100D4000CF0EBA16EE38300BBA12ED30F36EEF302C
:100D5000BB6EF332BB3217D842AE0BD0426A416A47
:100D6000406A3F6A206A00EE43F0240EEE68E82EE7
:100D7000FDD706D042AE04D0426A416A406A3F6A5B
:100D8000807411EF01F027686A8E116A090E115CF8
:100D900033E2D8901134E96EEA6AEA36E936EA3687
:100DA000430EE926000EEA22EFCF02F0ECCF03F06B
:100DB000ECCF04F0ECCF05F06750025C68500358AC
:100DC000695004586A50055815E2D8901134E96EFC
:100DD000EA6AEA36E936EA36430EE926000EEA22E6
:100DE000EFCF67F0ECCF68F0ECCF69F0ECCF6AF0B2
:100DF00011C027F0112ACAE31200220E175C0DE37E
:100E00002F0E175C0AE2A60EAEEC00F01750AEEC07
:100E100000F01850AEEC00F037D0470E175C0AE136
:100E2000A60EAEEC00F01750AEEC00F01850AEEC91
:100E300000F02AD07A0E175C03E118C022F024D00B
:100E4000780E175C03E118C023F01ED0790E175CF2
:100E500003E118C024F018D0150E175C15E13D6AA7
:100E600018C03CF0D8903C363D363C363D3600EE5E
:100E70003CF0CF0EBA16EE38300BBA12ED30F36EEE
:100E8000EF30BB6EF332BB3217681200150E195CDF
:100E900003E11AC03EF035D01E0E195C09E11FA017
:100EA00006D01AC022F01AC023F01AC024F029D0AC
:100EB000420E195C09E11A5204E18A941F9023D86A
:100EC00002D08A841F801DD07B0E195C1AE18A90A3
:100ED0008A928B908B968B988B9ACF0EBA16000EB7
:100EE000BA12000EBB6ECF0EBD16000EBD12000E64
:100EF000BE6E8998899A00EE43F0240EEE68E82EC3
:100F0000FDD7196812008998899A00EE43F0240EE3
:100F1000EE68E82EFDD78A94206A226A236A246A42
:100F20008A908A928B968B988B9A8B90CF0EBA165A
:100F3000000EBA12000EBB6ECF0EBD16000EBD1213
:100F4000000EBE6E1F6A010E3E6E3D6A3C6A1200C4
:100F500005016C696B695C0E6E6F7A0E6D6F590ED0
:100F6000706F850E6F6F580E726F140E716F560E84
:100F7000746FA90E736F550E766F430E756F530E17
:100F8000786FE30E776F520E7A6F890E796F510E7C
:100F90007C6F350E7B6F4F0E7E6FE60E7D6F4E0EB3
:100FA000806F9C0E7F6F4D0E826F580E816F4C0EBE
:100FB000846F190E836F4A0E866FDF0E856F490EA0
:100FC000886FAA0E876F480E8A6F7A0E896F470E58
:100FD0008C6F4F0E8B6F460E8E6F290E8D6F450EE8
:100FE000906F080E8F6F430E926FEB0E916F420E53
:100FF000946FD30E936F410E966FBF0E956F400E98
:10100000986FB00E976F3F0E9A6FA50E996F3E0EB8
:101010009C6F9E0E9B6F3D0E9E6F9C0E9D6F3C0EB7
:10102000A06F9E0E9F6F3B0EA26FA40EA16F3A0E93
:10103000A46FAE0EA36F390EA66FBC0EA56F380E4F
:10104000A86FCE0EA76F370EAA6FE30EA96F360EEC
:10105000AC6FFD0EAB6F360EAE6F1A0EAD6F350E68
:10106000B06F3B0EAF6F340EB26F5F0EB16F330EC9
:10107000B46F870EB36F320EB66FB20EB56F310E0E
:10108000B86FE10EB76F310EBA6F140EB96F300E34
:10109000BC6F490EBB6F2F0EBE6F820EBD6F2E0E42
:1010A000C06FBE0EBF6F2D0EC26FFD0EC16F2D0E35
:1010B000C46F3F0EC36F2C0EC66F850EC56F2B0E0F
:1010C000C86FCD0EC76F2B0ECA6F180EC96F2A0ED0
:1010D000CC6F670ECB6F290ECE6FB80ECD6F290E79
:1010E000D06F0C0ECF6F280ED26F620ED16F270E0D
:1010F000D46FBC0ED36F270ED66F180ED56F260E89
:10110000D86F760ED76F250EDA6FD80ED96F250EF1
:10111000DC6F3C0EDB6F240EDE6FA20EDD6F240E43
:10112000E06F0B0EDF6F230EE26F760EE16F220E83
:10113000E46FE40EE36F220EE66F540EE56F210EAE
:10114000E86FC60EE76F210EEA6F3B0EE96F200EC7
:10115000EC6FB20EEB6F200EEE6F2B0EED6F1F0ECD
:10116000F06FA60EEF6F1F0EF26F240EF16F1E0EC2
:10117000F46FA30EF36F1E0EF66F250EF56F1D0EA6
:10118000F86FA90EF76F1D0EFA6F2E0EF96F1C0E79
:10119000FC6FB60EFB6F1C0EFE6F3F0EFD6F1B0E3D
:1011A0000601006FCB0E0501FF6F1B0E0601026FDB
:1011B000580E016F1A0E046FE80E036F1A0E066FB9
:1011C000790E056F1A0E086F0B0E076F190E0A6F56
:1011D000A00E096F190E0C6F360E0B6F180E0E6FE6
:1011E000CE0E0D6F180E106F680E0F6F180E126F67
:1011F000030E116F170E146FA00E136F170E166FDC
:101200003F0E156F160E186FDF0E176F160E1A6F42
:10121000800E196F160E1C6F240E1B6F150E1E6F9D
:10122000C80E1D6F150E206F6E0E1F6F150E226FEC
:10123000160E216F140E246FBF0E236F140E266F2F
:10124000690E256F140E286F150E276F130E2A6F67
:10125000C20E296F130E2C6F710E2B6F130E2E6F93
:10126000210E2D6F120E306FD20E2F6F120E326FB5
:10127000840E316F120E346F380E336F110E366FCD
:10128000ED0E356F110E386FA30E376F110E3A6FDA
:101290005A0E396F110E3C6F120E3B6F100E3E6FDF
:1012A000CC0E3D6F100E406F870E3F6F100E426FD9
:1012B000420E416F0F0E446F4369466FBD0E456F7E
:1012C0000F0E486F7C0E476F0F0E4A6F3D0E496F31
:1012D0000E0E4C6FFE0E4B6F0E0E4E6FC00E4D6F0E
:1012E0000E0E506F830E4F6F0E0E526F470E516FE2
:1012F0000E0E546F0C0E536F0D0E566FD20E556FAF
:101300000D0E586F990E576F0D0E5A6F610E596F73
:101310000D0E5C6F2A0E5B6F0C0E5E6FF40E5D6F30
:101320000C0E606FBE0E5F6F0C0E626F8A0E616FE7
:101330000C0E646F560E636F0C0E666F230E656F96
:101340000B0E686FF10E676F0B0E6A6FC00E696F40
:101350006C696B69A20E6E6FC30E6D6F9A0E706F23
:10136000460E6F6F960E726F320E716F920E746F23
:101370003A0E736F8E0E766F5D0E756F8A0E786FF4
:101380009A0E776F860E7A6FF00E796F830E7C6FF0
:101390005F0E7B6F7F0E7E6FE70E7D6F7C0E806F22
:1013A000850E7F6F790E826F3B0E816F760E846F94
:1013B000070E836F720E866FE80E856F6F0E886F53
:1013C000DF0E876F6C0E8A6FEA0E896F6A0E8C6F64
:1013D0000A0E8B6F670E8E6F3C0E8D6F640E906FD2
:1013E000820E8F6F610E926FDA0E916F5F0E946FA7
:1013F000440E936F5C0E966FBF0E956F5A0E986FEA
:101400004C0E976F570E9A6FE90E996F550E9C6FA1
:10141000960E9B6F530E9E6F9D6F510EA06F200E08
:101420009F6F4E0EA26FFB0EA16F4C0EA46FE50EC8
:10143000A36F4A0EA66FDC0EA56F480EA86FE20ED2
:10144000A76F460EAA6FF50EA96F450EAC6F150E6D
:10145000AB6F430EAE6F420EAD6F410EB06F7B0EA1
:10146000AF6F3F0EB26FC00EB16F3E0EB46F100E75
:10147000B36F3C0EB66F6D0EB56F3A0EB86FD40EEB
:10148000B76F390EBA6F460EB96F370EBC6FC20E0A
:10149000BB6F360EBE6F490EBD6F340EC06FDA0ED5
:1014A000BF6F330EC26F740EC16F320EC46F180E51
:1014B000C36F300EC66FC50EC56F2F0EC86F7B0E83
:1014C000C76F2E0ECA6F3A0EC96F2D0ECC6F020E6B
:1014D000CB6F2B0ECE6FD10ECD6F2A0ED06FA90E13
:1014E000CF6F290ED26F880ED16F280ED46F6F0E7A
:1014F000D36F270ED66F5E0ED56F260ED86F530EA4
:10150000D76F250EDA6F500ED96F240EDC6F540E94
:10151000DB6F230EDE6F5E0EDD6F220EE06F6F0E4F
:10152000DF6F210EE26F860EE16F200EE46FA30ED7
:10153000E36F1F0EE66FC60EE56F1E0EE86FEF0E2F
:10154000E76F1E0EEA6FE96F1D0EEC6F520EEB6F28
:101550001C0EEE6F8C0EED6F1B0EF06FCB0EEF6F4F
:101560001B0EF26F0F0EF16F1A0EF46F580EF36F21
:10157000190EF66FA50EF56F180EF86FF80EF76FCF
:10158000180EFA6F4F0EF96F170EFC6FAB0EFB6F54
:10159000170EFE6F0A0EFD6F160E0701006F6F0E1D
:1015A0000601FF6F150E0701026FD70E016F150EB2
:1015B000046F430E036F140E066FB30E056F140E07
:1015C000086F270E076F130E0A6F9F0E096F130E19
:1015D0000C6F1A0E0B6F120E0E6F990E0D6F120E0E
:1015E000106F1B0E0F6F110E126FA10E116F110EE7
:1015F000146F290E136F100E166FB50E156F100EA7
:10160000186F440E176F0F0E1A6FD60E196F0F0E4C
:101610001C6F6B0E1B6F0F0E1E6F030E1D6F0E0ED9
:10162000206F9D0E1F6F0E0E226F3A0E216F0D0E52
:10163000246FDA0E236F0D0E266F7C0E256F0D0EB4
:10164000286F210E276F0C0E2A6FC80E296F0C0E03
:101650002C6F720E2B6F0C0E2E6F1E0E2D6F0B0E3D
:10166000306FCC0E2F6F0B0E326F7C0E316F0B0E66
:10167000346F2E0E336F0A0E366FE30E356F0A0E7F
:10168000386F990E376F0A0E3A6F510E396F0A0E86
:101690003C6F0B0E3B6F090E3E6FC80E3D6F090E7F
:1016A000406F850E3F6F090E426F450E416F090E68
:1016B000446F060E436F080E466FC90E456F080E45
:1016C000486F8E0E476F080E4A6F540E496F080E12
:1016D0004C6F1C0E4B6F070E4E6FE50E4D6F070ED5
:1016E000506FAF0E4F6F070E526F7B0E516F070E8C
:1016F000546F490E536F070E566F170E556F060E37
:10170000586FE70E576F060E5A6FB90E596F060ED7
:101710005C6F8B0E5B6F060E5E6F5F0E5D6F060E6D
:10172000606F340E5F6F060E626F0A0E616F050EFA
:10173000646FE10E636F050E666FB90E656F050E7F
:10174000686F930E676F050E6A6F6D0E696F00010B
:101750001200040E01016E6F880E6D6F040E706F23
:10176000A60E6F6F040E726FB60E716F040E746F5B
:10177000C60E736F040E766FD60E756F040E786FFB
:10178000E60E776F040E7A6FF60E796F050E7C6F9A
:10179000070E7B6F050E7E6F170E7D6F050E806F37
:1017A000280E7F6F050E826F390E816F050E846FD4
:1017B0004B0E836F050E866F5D0E856F050E886F6D
:1017C0006E0E876F050E8A6F800E896F050E8C6F07
:1017D000930E8B6F050E8E6FA50E8D6F050E906F9D
:1017E000B80E8F6F050E926FCB0E916F050E946F32
:1017F000DF0E936F050E966FF20E956F060E986FC3
:10180000976F9A6F1A0E996F060E9C6F2E0E9B6F34
:10181000060E9E6F430E9D6F060EA06F580E9F6FB3
:10182000060EA26F6D0EA16F060EA46F830EA36F3E
:10183000060EA66F980EA56F060EA86FAE0EA76FC8
:10184000060EAA6FC40EA96F060EAC6FDB0EAB6F4F
:10185000060EAE6FF20EAD6F070EB06F090EAF6FD2
:10186000070EB26F210EB16F070EB46F380EB36F53
:10187000070EB66F500EB56F070EB86F690EB76FD3
:10188000070EBA6F810EB96F070EBC6F9A0EBB6F51
:10189000070EBE6FB40EBD6F070EC06FCD0EBF6FCB
:1018A000070EC26FE70EC16F080EC46F020EC36F42
:1018B000080EC66F1D0EC56F080EC86F380EC76FB5
:1018C000080ECA6F530EC96F080ECC6F6F0ECB6F28
:1018D000080ECE6F8B0ECD6F080ED06FA70ECF6F98
:1018E000080ED26FC40ED16F080ED46FE10ED36F05
:1018F000080ED66FD569090ED86F1D0ED76F090E69
:10190000DA6F3B0ED96F090EDC6F5A0EDB6F090ED2
:10191000DE6F790EDD6F090EE06F990EDF6F090E35
:10192000E26FB90EE16F090EE46FD90EE36F090E95
:10193000E66FFA0EE56F0A0EE86F1B0EE76F0A0EF0
:10194000EA6F3D0EE96F0A0EEC6F5F0EEB6F0A0E49
:10195000EE6F820EED6F0A0EF06FA50EEF6F0A0E9E
:10196000F26FC80EF16F0A0EF46FEC0EF36F0B0EF0
:10197000F66F110EF56F0B0EF86F360EF76F0B0E3C
:10198000FA6F5B0EF96F0B0EFC6F810EFB6F0B0E87
:10199000FE6FA70EFD6F0B0E0201006FCE0E010150
:1019A000FF6F0B0E0201026FF50E016F0C0E046F3C
:1019B0001D0E036F0C0E066F460E056F0C0E086FA2
:1019C0006F0E076F0C0E0A6F980E096F0C0E0C6FDE
:1019D000C20E0B6F0C0E0E6FED0E0D6F0D0E106F15
:1019E000180E0F6F0D0E126F430E116F0D0E146F48
:1019F000700E136F0D0E166F9C0E156F0D0E186F77
:101A0000CA0E176F0D0E1A6FF80E196F0E0E1C6F9F
:101A1000260E1B6F0E0E1E6F550E1D6F0E0E206FC5
:101A2000850E1F6F0E0E226FB60E216F0E0E246FE5
:101A3000E70E236F0F0E266F180E256F0F0E286FFF
:101A40004B0E276F0F0E2A6F7E0E296F0F0E2C6F15
:101A5000B10E2B6F0F0E2E6FE60E2D6F100E306F26
:101A60001B0E2F6F100E326F500E316F100E346F31
:101A7000870E336F100E366FBE0E356F100E386F37
:101A8000F60E376F110E3A6F2E0E396F110E3C6F36
:101A9000680E3B6F110E3E6FA20E3D6F110E406F30
:101AA000DC0E3F6F120E426F180E416F120E446F24
:101AB000540E436F120E466F910E456F120E486F13
:101AC000CF0E476F130E4A6F0E0E496F130E4C6FF9
:101AD0004D0E4B6F130E4E6F8E0E4D6F130E506FDB
:101AE000CF0E4F6F140E526F110E516F140E546FB4
:101AF000540E536F140E566F980E556F140E586F88
:101B0000DC0E576F150E5A6F220E596F150E5C6F53
:101B1000680E5B6F150E5E6FB00E5D6F150E606F19
:101B2000F80E5F6F160E626F410E616F160E646FD6
:101B30008C0E636F160E666FD70E656F170E686F8B
:101B4000230E676F170E6A6F700E696F116A0001BE
:101B5000800E115C3CE201EE6BF0D8901134E92666
:101B6000000EEA22EECF06F0EFCF07F0D890073054
:101B7000036E0630026E02EE6BF0D8901134E92647
:101B8000000EEA2202C0EEFF03C0EFFF01EE6BF091
:101B9000D8901134E926000EEA22EECF06F0EFCFFE
:101BA00007F0D8900730036E0630026ED8900332EB
:101BB000023203EE6BF0D8901134E926000EEA22CF
:101BC00002C0EEFF03C0EFFF112AD8A0C0D7020E5B
:101BD00004016C6F940E6B6F010E116E0001800E8C
:101BE000115C1DE26BC406F06CC407F01150060DC9
:101BF000F3CF0EF0F4CF0FF00E500624026E0F500C
:101C00000720036E04EE6BF0D8901134E926000E25
:101C1000EA2202C0EEFF03C0EFFF112ADFE3120049
:101C200008016E6B020E6D6F07016E6B300E6D6FEB
:101C30000801706B020E6F6F0701706B300E6F6FD3
:101C40000801726B020E716F0701726B300E716FBB
:101C50000801746B020E736F0701746B170E736FBC
:101C60000801766B020E756F0701766B170E756FA4
:101C70000801786B020E776F0701786B170E776F8C
:101C800008017A6B020E796F07017A6B170E796F74
:101C900008017C6B020E7B6F07017C6B170E7B6F5C
:101CA00008017E6B020E7D6F07017E6B170E7D6F44
:101CB0000801806B060E7F6F0701806B2C0E7F6F13
:101CC0000801826B060E816F0701826B2C0E816FFB
:101CD0000801846B060E836F0701846B2C0E836FE3
:101CE0000801866B060E856F0701866B2C0E856FCB
:101CF0000801886B060E876F0701886B2C0E876FB3
:101D000008018A6B040E896F07018A6B150E896FB3
:101D100008018C6B040E8B6F07018C6B150E8B6F9B
:101D200008018E6B040E8D6F07018E6B150E8D6F83
:101D30000801906B040E8F6F0701906B150E8F6F6B
:101D40000801926B040E916F0701926B150E916F53
:101D50000801946B0A0E936F0701946B280E936F22
:101D60000801966B0A0E956F0701966B280E956F0A
:101D70000801986B0A0E976F0701986B280E976FF2
:101D800008019A6B0A0E996F07019A6B280E996FDA
:101D900008019C6B0A0E9B6F07019C6B280E9B6FC2
:101DA00008019E6B060E9D6F07019E6B130E9D6FC3
:101DB0000801A06B060E9F6F0701A06B130E9F6FAB
:101DC0000801A26B060EA16F0701A26B130EA16F93
:101DD0000801A46B060EA36F0701A46B130EA36F7B
:101DE0000801A66B060EA56F0701A66B130EA56F63
:101DF0000801A86B060EA76F0701A86B130EA76F4B
:101E00000801AA6B0E0EA96F0701AA6B240EA96F19
:101E10000801AC6B0E0EAB6F0701AC6B240EAB6F01
:101E20000801AE6B0E0EAD6F0701AE6B240EAD6FE9
:101E30000801B06B0E0EAF6F0701B06B240EAF6FD1
:101E40000801B26B0E0EB16F0701B26B240EB16FB9
:101E50000801B46B080EB36F0701B46B110EB36FBA
:101E60000801B66B080EB56F0701B66B110EB56FA2
:101E70000801B86B080EB76F0701B86B110EB76F8A
:101E80000801BA6B080EB96F0701BA6B110EB96F72
:101E90000801BC6B080EBB6F0701BC6B110EBB6F5A
:101EA0000801BE6B120EBD6F0701BE6B200EBD6F29
:101EB0000801C06B120EBF6F0701C06B200EBF6F11
:101EC0000801C26B120EC16F0701C26B200EC16FF9
:101ED0000801C46B120EC36F0701C46B200EC36FE1
:101EE0000801C66B120EC56F0701C66B200EC56FC9
:101EF0000801C86B0A0EC76F0701C86B0F0EC76FCA
:101F00000801CA6B0A0EC96F0701CA6B0F0EC96FB1
:101F10000801CC6B0A0ECB6F0701CC6B0F0ECB6F99
:101F20000801CE6B0A0ECD6F0701CE6B0F0ECD6F81
:101F30000801D06B0A0ECF6F0701D06B0F0ECF6F69
:101F40000801D26B0A0ED16F0701D26B0F0ED16F51
:101F50000801D46B160ED36F0701D46B1C0ED36F20
:101F60000801D66B160ED56F0701D66B1C0ED56F08
:101F70000801D86B160ED76F0701D86B1C0ED76FF0
:101F80000801DA6B160ED96F0701DA6B1C0ED96FD8
:101F90000801DC6B160EDB6F0701DC6B1C0EDB6FC0
:101FA0000801DE6B0C0EDD6F0701DE6B0D0EDD6FC1
:101FB0000801E06B0C0EDF6F0701E06B0D0EDF6FA9
:101FC0000801E26B0C0EE16F0701E26B0D0EE16F91
:101FD0000801E46B0C0EE36F0701E46B0D0EE36F79
:101FE0000801E66B0C0EE56F0701E66B0D0EE56F61
:101FF0000801E86B1A0EE76F0701E86B180EE76F30
:102000000801EA6B1A0EE96F0701EA6B180EE96F17
:102010000801EC6B1A0EEB6F0701EC6B180EEB6FFF
:102020000801EE6B1A0EED6F0701EE6B180EED6FE7
:102030000801F06B1A0EEF6F0701F06B180EEF6FCF
:102040000801F26B0E0EF16F0701F26B0B0EF16FD0
:102050000801F46B0E0EF36F0701F46B0B0EF36FB8
:102060000801F66B0E0EF56F0701F66B0B0EF56FA0
:102070000801F86B0E0EF76F0701F86B0B0EF76F88
:102080000801FA6B0E0EF96F0701FA6B0B0EF96F70
:102090000801FC6B0E0EFB6F0701FC6B0B0EFB6F58
:1020A0000801FE6B1E0EFD6F0701FE6B140EFD6F27
:1020B0000901006B1E0E0801FF6F006B140E070173
:1020C000FF6F0901026B1E0E016F0801026B140EF7
:1020D000016F0901046B1E0E036F0801046B140EDF
:1020E000036F0901066B1E0E056F0801066B140EC7
:1020F000056F0901086B100E076F0801086B090EC8
:10210000076F09010A6B100E096F08010A6B090EAF
:10211000096F09010C6B100E0B6F08010C6B090E97
:102120000B6F09010E6B100E0D6F08010E6B090E7F
:102130000D6F0901106B100E0F6F0801106B090E67
:102140000F6F0901126B220E116F0801126B100E36
:10215000116F0901146B220E136F0801146B100E1E
:10216000136F0901166B220E156F0801166B100E06
:10217000156F0901186B220E176F0801186B100EEE
:10218000176F09011A6B220E196F08011A6B100ED6
:10219000196F09011C6B120E1B6F08011C6B070ED7
:1021A0001B6F09011E6B120E1D6F08011E6B070EBF
:1021B0001D6F0901206B120E1F6F0801206B070EA7
:1021C0001F6F0901226B120E216F0801226B070E8F
:1021D000216F0901246B120E236F0801246B070E77
:1021E000236F0901266B120E256F0801266B070E5F
:1021F000256F0901286B260E276F0801286B0C0E2E
:10220000276F09012A6B260E296F08012A6B0C0E15
:10221000296F09012C6B260E2B6F08012C6B0C0EFD
:102220002B6F09012E6B260E2D6F08012E6B0C0EE5
:102230002D6F0901306B260E2F6F0801306B0C0ECD
:102240002F6F0901326B140E316F0801326B050ECE
:10225000316F0901346B140E336F0801346B050EB6
:10226000336F0901366B140E356F0801366B050E9E
:10227000356F0901386B140E376F0801386B050E86
:10228000376F09013A6B140E396F08013A6B050E6E
:10229000396F09013C6B2A0E3B6F08013C6B080E3D
:1022A0003B6F09013E6B2A0E3D6F08013E6B080E25
:1022B0003D6F0901406B2A0E3F6F0801406B080E0D
:1022C0003F6F0901426B2A0E416F0801426B080EF5
:1022D000416F0901446B2A0E436F0801446B080EDD
:1022E000436F0901466B160E456F0801466B030EDE
:1022F000456F0901486B160E476F0801486B030EC6
:10230000476F09014A6B160E496F08014A6B030EAD
:10231000496F09014C6B160E4B6F08014C6B030E95
:102320004B6F09014E6B160E4D6F08014E6B030E7D
:102330004D6F0901506B160E4F6F0801506B030E65
:102340004F6F0901526B2E0E516F0801526B040E34
:10235000516F0901546B2E0E536F0801546B040E1C
:10236000536F0901566B2E0E556F0801566B040E04
:10237000556F0901586B2E0E576F0801586B040EEC
:10238000576F09015A6B2E0E596F08015A6B040ED4
:10239000596F09015C6B180E5B6F08015C6B010ED5
:1023A0005B6F09015E6B180E5D6F08015E6B010EBD
:1023B0005D6F0901606B180E5F6F0801606B010EA5
:1023C0005F6F0901626B180E616F0801626B010E8D
:1023D000616F0901646B180E636F0801646B010E75
:1023E000636F0901666B320E656F0801666B656B82
:1023F0000901686B676F0801686B676B010E116EEE
:1024000000017F0E115CD8B04BD008EE6BF0D89075
:102410001134E926000EEA22EECF06F0EFCF07F0E6
:102420000650E80DF3CF02F0F4CF03F00750E80DAB
:10243000F35003260650030DF350032608EE6BF00D
:10244000D8901134E926000EEA2202C0EEFF03C044
:10245000EFFF07EE6BF0D8901134E926000EEA2268
:10246000EECF06F0EFCF07F00650E80DF3CF02F005
:10247000F4CF03F00750E80DF35003260650030D88
:10248000F350032607EE6BF0D8901134E926000EC6
:10249000EA2202C0EEFF03C0EFFF112AD8A0B0D796
:0424A0001200FFD750
:020000040030CA
:0300010006160ED2
:020005008580F4
:060008000FC00FE00F40E5
:00000001FF
